:020000040800F2
:10000000300C0024AD020008EF3500088B2E0008EC
:10001000B90200089503000815450008000000001B
:10002000000000000000000000000000FD3A000891
:10003000BB04000800000000F1350008FD3C00088A
:10004000C7020008C7020008C7020008C70200086C
:10005000C7020008C7020008C7020008C70200085C
:10006000C7020008C7020008C7020008C70200084C
:10007000C7020008C7020008C7020008C70200083C
:10008000C7020008C7020008C7020008C70200082C
:10009000C7020008C7020008C7020008C70200081C
:1000A000C7020008C7020008C7020008C70200080C
:1000B000C7020008C7020008C7020008C7020008FC
:1000C000C7020008C7020008C7020008C7020008EC
:1000D000C7020008D1440008C7020008C702000890
:1000E000C7020008C702000800000000C70200089D
:1000F000C7020008C7020008C7020008C7020008BC
:10010000C7020008C7020008C7020008C7020008AB
:10011000C7020008C7020008C7020008C70200089B
:10012000C7020008C7020008C7020008C70200088B
:10013000C7020008C7020008C7020008C70200087B
:1001400000000000000000000000000000000000AF
:10015000C7020008C7020008C7020008C70200085B
:10016000C7020008C7020008C7020008C70200084B
:10017000C7020008C7020008C7020008C70200083B
:10018000C7020008C7020008C7020008C70200082B
:10019000C7020008C7020008C7020008C70200081B
:1001A000C7020008C7020008C7020008C70200080B
:1001B000C7020008C7020008C7020008C7020008FB
:1001C000C7020008C7020008C7020008C7020008EB
:1001D000C7020008C7020008C7020008C7020008DB
:1001E000C7020008C7020008C7020008C7020008CB
:1001F000C7020008C7020008C7020008C7020008BB
:10020000C7020008C7020008C7020008C7020008AA
:10021000C7020008C7020008C7020008C70200089A
:10022000C7020008C7020008C7020008000000005B
:10023000C7020008C702000800000000C70200084B
:10024000C7020008C7020008C7020008C70200086A
:10025000C7020008C7020008C7020008C70200085A
:10026000C7020008C7020008C7020008C70200084A
:10027000C7020008C7020008C7020008000000000B
:10028000C702000800000000C702000800000000CC
:1002900000000000C7020008DFF80CD000F068F88A
:1002A00000480047B9450008300C00240648804744
:1002B00006480047FEE7FEE7FEE7FEE7FEE7FEE74B
:1002C000FEE7FEE7FEE7FEE7013D000899020008B1
:1002D0002DE9F05F0546002092469B46884606467B
:1002E000814640241BE0284641464746224600F00E
:1002F0002FF853465A46C01A914110D3114618465A
:10030000224600F016F82D1A67EB01084F462246E8
:100310000120002100F00DF817EB00094E41201ECE
:10032000A4F10104DFDC484631462A464346BDE8D5
:10033000F09F202A04DB203A00FA02F100207047E7
:100340009140C2F1200320FA03F319439040704713
:10035000202A04DB203A21FA02F00021704721FA1A
:1003600002F3D040C2F12002914008431946704781
:10037000064C074D06E0E06840F0010394E80700F2
:1003800098471034AC42F6D3FFF78AFF886A00081A
:10039000A86A0008FEE70000F0B5BFF34F8FBFF377
:1003A0006F8F1D4900200860BFF34F8FBFF36F8F21
:1003B0001A4C216841F400312160BFF34F8FBFF325
:1003C0006F8F164970310860BFF34F8F081F0068A8
:1003D00043F6FF75104E1036C0F34E31C0F3C9031B
:1003E00005EA4112184642EA80773760401EFAD289
:1003F000491EF5D2BFF34F8F206840F48030206053
:10040000BFF34F8FBFF36F8F03484C30016841F04B
:1004100004010160F0BD000050EF00E014ED00E0C9
:100420002DE9F0430D4F00241D46164688468146AF
:1004300004EB041017F81010B14209D107EB40018A
:100440004878A84204D1891C4246484600F02AF860
:10045000641CA4B2382CEBD3BDE8F083CE5F000857
:100460002DE9F0430E4F00241D461646884681466E
:1004700004EB840000EB441017F81010B14209D1CE
:1004800007EB40014878A84204D1891C42464846FF
:1004900000F008F8641CA4B2092CE9D3BDE8F0838D
:1004A000A4670008002310B504E011F8014B5B1CA1
:1004B00000F8014B9342F8D310BD7047F0B51C46CD
:1004C000094B0A4F164685B04FF0000C10251A88CC
:1004D0005B883F88121A5B1A8DE8F01092B29BB2CB
:1004E00000F008FB05B0F0BD1C0200242C00002425
:1004F0002DE9FF411C46084B1646002710251A8897
:100500005B88121A5B1A8DE8F00092B29BB203F07E
:1005100043FBBDE8FF8100001C02002470B51A4BAC
:10052000CC074FF4E06513D0DC6824F4E664DC60AB
:10053000DC6895FAA5F6B6FA86F6144300FA06F6D4
:1005400046F004063443DC60DC6844F08004DC6080
:10055000890718D5D3F80C1121F4E661C3F80C1102
:10056000D3F80C11114395FAA5F2B2FA82F2904039
:1005700040F004000143C3F80C11D3F80C0140F023
:100580008000C3F80C0170BD00200052CA4340F047
:1005900008009307174A20D0CB070AD0D36823F06E
:1005A0003003D360D3680343D360D36843F0800340
:1005B000D360890710D5D2F80C1121F03001C2F8B0
:1005C0000C11D2F80C110143C2F80C11D2F80C0135
:1005D00040F08000C2F80C017047D16821F0300172
:1005E000D160D1680143D160906940F0080090610A
:1005F00070470000002000524A4900228A61012809
:10060000494A2ED002287DD1D2F81001800303D5AB
:10061000886940F480508861D2F81001400303D506
:10062000886940F400508861D2F81001000303D5B6
:10063000886940F480408861D2F81001800203D5B7
:10064000886940F400408861D2F81001400203D567
:10065000886940F4803088611369344898433FD0FA
:1006600042E01069800303D5886940F00100886189
:100670001069400303D5886940F002008861106961
:10068000000303D5886940F0040088611069800286
:1006900003D5886940F0080088611069400203D5DD
:1006A000886940F0100088611069000203D58869EC
:1006B00040F0200088611069C00103D5886940F0CE
:1006C000400088611069800103D5886940F080008E
:1006D00088611069400123D5886940F480701EE06C
:1006E000886940F40030886113694FF001409843F5
:1006F00003D1886940F48020886113694FF002407B
:10070000984300E00CE003D1886940F40020886140
:10071000D2F81001400103D5886940F48010886147
:100720007047000078010024002000520000808003
:100730002DE9F05F00250F46804600F0D3FC254EE2
:1007400000EB080A224C012FB06902D1002800DB1F
:100750000724DFF884B004EA0B09B9F1000F14D0C4
:10076000D6F8100124EA0000400020B1012F10D07B
:10077000022F14D01BE0B8F1FF3FEED000F0B2FC26
:100780005045EAD30320BDE8F09F306924EA000019
:10079000EBE730691149084209D00D4608E0D6F868
:1007A00010110F480140490001D0054600E06DB12D
:1007B0003846FFF721FF15EA0B0F01D1756103E001
:1007C00025F00040C6F814010120DCE70020DAE73C
:1007D0000700008000200052F0FF10F00000EE073C
:1007E0000000EE872DE9F0411546DFF85C8001221C
:1007F0000C46064640461703394600F06EFC0520BD
:1008000000F0D6F9032003F013F8C4F3074003F017
:100810000FF8C4F3072003F00BF8E0B203F008F878
:10082000002405E0FF2003F003F83055641CA4B257
:10083000AC42F7D300223946404600F04EFCBDE8FA
:10084000F041052000F0B4B90004025830B40C4661
:100850000178202A1AD009DC0C2A0DD0102A13D0D6
:10086000182A17D10C4801FB030108E0302A0FD0E9
:10087000402A0FD10948F6E7594301F500212046E7
:1008800030BC1A46FFF7AEBF0548ECE70548EAE77B
:100890000548E8E730BC70470012080000920800E5
:1008A00000080800002608000048080030B40C4684
:1008B0000146007815464A78812809D3402A07D393
:1008C000FF2A05D0FF2803D07F2A0CD2403A0BE044
:1008D0000022104603E0521C92B204F8010B9A4227
:1008E000F9D330BC7047413A8138C0B2D1B2C0EBC5
:1008F000401202EB801001EB400159430C2D0CD04B
:10090000102D0CD0182D0DD0202DEAD101F560113D
:10091000204630BC1A46FFF765BF044800E0044893
:100920000144F5E701F5ED11F2E7000000140900BC
:1009300000DD1100AFF3008070B586B04FF6FF7098
:1009400002F016FB00206C4605462554401CC0B240
:100950001828FAD3112220460021FFF743FF102167
:100960006B464FF4784608463246FFF7A7FD002055
:100970002554401CC0B21828FAD308226846142116
:10098000FFF730FF20216B4610203246FFF796FD1F
:1009900000202554401CC0B21828FAD3082268460B
:1009A0001E21FFF71FFF30216B4610203246FFF754
:1009B00085FD4FF4FA6003F0D7FD06B070BD2DE958
:1009C000F04FC1B01C4616460D4682468946580770
:1009D00001D0012100E0002101EBD40061080C2CC2
:1009E00010FB01F0834609D0102C07D0182C05D03D
:1009F000202C03D0302C01D0402C2DD10346224690
:100A000069463046FFF722FF002022E01DF80870FB
:100A10000026380601D54A9A02E04C9820B94B9A34
:100A20002946504602F006FB78066D1CADB2070E53
:100A3000A5EB0900A04205D10AF101004D461FFABD
:100A400080FA03E0761CB6B2082EE2D308F101006A
:100A500080B258458046D9D341B0BDE8F08F2DE92A
:100A6000F04FA1B01F4615460C46824689465807EE
:100A700001D0012100E0002101EBD7000C2F10FB79
:100A800007F0834605D0102F03D0182F01D0202F58
:100A90002DD103463A4669462846FFF707FF002056
:100AA00022E01DF808600025300601D52A9A02E0F0
:100AB0002C9820B92B9A2146504602F0BBFA7006BA
:100AC000641CA4B2060EA4EB0900B84205D10AF1D9
:100AD00001004C461FFA80FA03E06D1CEDB2082DB0
:100AE000E2D308F10100C0B258458046D9D321B005
:100AF000BDE8F08F2DE9FF4F83B09B460E460446BC
:100B000080468A46DDE910750020814620E0B9F173
:100B1000000F23D005994FF0000908EB0100401B9E
:100B2000A04202DA7019444686B20AEB0B00401B61
:100B3000B04210DB12AB93E807002B468DE80700AC
:100B40003A4631462046FFF78AFF601984B2BF1C3F
:100B500038780028DBD107B0BDE8F08F802801D9B4
:100B60000120D2E7059A08EB0201A1EB5501A14251
:100B700002DA711944468EB20AEB0B01491BB142ED
:100B8000E9DB0D280FD012AB93E807002B468DE868
:100B900007003A4631462046FFF711FF04EB5500A7
:100BA00084B27F1CD4E77019444686B27F1CF5E7F7
:100BB000002206E00021491CC9B26429FBD3521C63
:100BC000D2B28242F6D3704770B4164602781D4600
:100BD0004378812A0C4610D3402B0ED3FF2B0CD028
:100BE000FF2A0AD00C2D11D0102D11D0182D0DD1A7
:100BF0003146204670BCFFF733BC0021084603E0B5
:100C0000491C04F8010BC9B2B142F9D370BC70475A
:100C10003146204670BCFFF703BC000010B528B178
:100C200090F83510022903D080214165012010BDC4
:100C30001D4A4FF4956301688C189C4207D8042222
:100C400080F83520086820F00100086029E00C6871
:100C500024F00E040C6001680A440A6822F00102C4
:100C60000A60016E0A6822F480720A6090F85C30B3
:100C7000012202FA03F10D4B1960D0E919134B6000
:100C8000C16E31B10B6823F480730B60D0E91C1383
:100C90004B60002180F8341080F83520016D01B1DF
:100CA0008847002010BD0000F0FFFDBF045402582B
:100CB0000248016841F001010160704720040058BA
:100CC0002DE9F05F04463C4889460025017D012955
:100CD00015D001210175824620794CF2503BC007A6
:100CE00003D05846FFF724FD05462079800704D538
:100CF00002215846FFF71CFD05431DB156E00220B6
:100D0000BDE8F09F4FF0FF31C9F8001020682B4F6D
:100D1000012803D0A66840F2047842E061682069A7
:100D2000FFF734FC2079C00708D001215846FFF7AF
:100D3000FFFC0546F86820F00800F860207980077D
:100D400034D502215846FFF7F3FC0543D7F80C01D0
:100D500020F00800C7F80C0128E0226930466168DD
:100D6000FFF7DCFB2079C00708D001215846FFF7C8
:100D7000DFFC0546F86820EA0800F8602079800763
:100D80000AD502215846FFF7D3FC0546D7F80C01D7
:100D900020EA0800C7F80C0115B1C9F8006005E0A9
:100DA000761CD4E902100844B042D6D80021284667
:100DB0008AF81410A4E700007801002400200052F3
:100DC0000648C16841F00101C160D0F80C1141F042
:100DD0000101C0F80C1100207047000000200052F3
:100DE0002F482DE9F0471546027D04260C46012ABE
:100DF00009D001228146A4F100610275B1F5003FDE
:100E000004D2012703E00220BDE8F08702274CF25C
:100E1000503A39465046FFF78BFC70BBDFF88880AC
:100E2000012F204940462CD0C0F81411D0F80C11E5
:100E300041F00201C0F80C11286869682060616007
:100E400008340835761E16F0FF06F5D1BFF34F8F34
:100E500039465046FFF76CFC012F41464FF4803273
:100E600015D0D1F81031DB0301D5C1F81421D1F828
:100E70000C2122F00202C1F80C21002289F8142072
:100E8000C2E74161C16841F00201C160D4E70B696A
:100E9000DB0300D54A61CA6822F00202CA60ECE7AF
:100EA000780100240600EF07002000520948C168BD
:100EB000C9070DD0D0F80C11C90709D00649416007
:100EC000064A4260C0F80411C0F8042100207047AF
:100ED000012070470020005223016745AB89EFCD08
:100EE0002DE9F84F6C4C00224FF0B04A4FF0010B47
:100EF0004FF0030E4FF00F090B680BFA02F73B405F
:100F0000BB4270D14D68022D01D0122D12D1D508EF
:100F100000EB850CDCF820605507ED0E09FA05F8AA
:100F200026EA0806D1F8108008FA05F848EA06080B
:100F3000CCF82080D0F80080560091F804C00EFA5A
:100F400006F50CF0030C28EA05080CFA06FC4CEA3E
:100F5000080CC0F800C0D1F804C0BCF1010F08D0E3
:100F6000BCF1020F05D0BCF1110F02D0BCF1120F81
:100F700016D1D0F808C0D1F80C802CEA050C08FA7C
:100F800006F848EA0C08C0F80880D0F804C02CEA3B
:100F9000070C0F79C7F30017974047EA0C07476023
:100FA000C768AF438D68B5403D43C5604D68ED00EF
:100FB0006BD53A4D2E6846F002062E602D6822F061
:100FC000030606F1B04605F002050095D6F808C400
:100FD00095072F0F09FA07F52CEA050C304DA842AA
:100FE00002D100252EE050E02E4DA84201D101256E
:100FF00028E02D4DA84201D1022523E02B4DA84227
:1010000001D103251EE02A4DA84201D1042519E093
:10101000284DA84201D1052514E0274DA84201D151
:1010200006250FE0254DA84201D107250AE0244DF1
:10103000A84201D1082505E0224DA84201D1092589
:1010400000E00A25BD4045EA0C05C6F808542568AD
:101050004E689D43F60300D51D43256065684E68C4
:101060009D43B60300D51D436560DAF8005056462F
:101070004F689D43FF0200D51D43356075684F687A
:101080009D43BF0200D51D437560521C102AFFF41A
:1010900033AFBDE8F88F000080000058F4440258D8
:1010A000000002580004025800080258000C0258C0
:1010B000001002580014025800180258001C025870
:1010C00000200258002402580069084000D0012086
:1010D000704742694A40426170470AB101837047D4
:1010E0004183704701488068704700001C0000245D
:1010F0000248816802781144816070471C00002416
:10110000032010B500F0A2F80F2000F007F808B196
:10111000012010BD00F06CF8002010BD70B50D4D21
:1011200004464FF47A712878B1FBF0F00A49096857
:10113000B1FBF0F001F0D6FC48B9102C07D2002228
:101140002146501E00F062F800206C6070BD012046
:1011500070BD00001C0000240C000024134A4178DC
:101160001160111D03780A1DE3B143680B60017B18
:10117000C37A090741EA0361837A41EAC341437BA9
:1011800041EA8341837B41EA4341C37B41EA034116
:10119000437A41EA0321037A007841EA430101439B
:1011A00011607047002008601060704798ED00E003
:1011B000BFF35F8F0448016821F480310160024968
:1011C000002070310860704724ED00E0074940F0CE
:1011D0000100086005487038016841F48031016001
:1011E000BFF34F8FBFF36F8F7047000094ED00E0A7
:1011F0007047002809DB012100F01F0291404009DF
:10120000800000F1E020C0F8001170470E4BF0B4F0
:101210001B68C3F30223C3F10704042C00D9042480
:101220001D1D072D01D2002300E0DB1E012606FA5A
:1012300004F56D1E0D409D409E40761E164045EA09
:101240000601F0BC03F067B90CED00E0064A00F0BF
:10125000070110684FF6FF03184040EA01200349D8
:1012600008431060704700000CED00E00000FA0534
:1012700010B500F0B3FE084909684FF4807292FA85
:10128000A2F201F47061B2FA82F2D140034A515CD9
:10129000C8400349086010BD18440258E5470008DB
:1012A0000C00002410B500F053FE07490968102215
:1012B00092FAA2F201F07001B2FA82F2D140034A2E
:1012C000515CC84010BD000020440258E5470008AA
:1012D000364930B50A68096812F00302344BC1F38D
:1012E00005311B68334C03F010032468DFED320A2C
:1012F000B7EE001AC4F3CC0414FB03F300EE103A6B
:101300002E4BB8EE400A07D02D4C012A01D0022AFC
:101310004AD0B4FBF1F10BE0244C283C226895063E
:10132000284A03D52468C4F3C104E240B2FBF1F1BA
:1013300001EE901A1968B8EE612AC1F3080101EEB6
:10134000901A1968F8EE611A40EE201A31EE810AFF
:1013500022EE000AC1F34621491C00EE901AF8EE75
:10136000600A80EE201AFCEEC10AC0ED000A19687E
:10137000C1F30641491C00EE901AF8EE600A80EEB7
:10138000201AFCEEC10AC0ED010A1968C1F306611A
:10139000491C00EE901AF8EE600A80EE201ABCEEAE
:1013A000C10A80ED020A30BD074ABFE7284402584F
:1013B0002C4402583C44025800000039384402587A
:1013C00000093D000090D00340787D01364930B5DA
:1013D0000A68096812F00302344BC1F305511B6817
:1013E000334C03F480732468DFED320AB7EE001A41
:1013F000C4F3CC0414FB03F300EE103A2E4BB8EE0A
:10140000400A07D02D4C012A01D0022A4AD0B4FB51
:10141000F1F10BE0244C283C22689506284A03D5BC
:101420002468C4F3C104E240B2FBF1F101EE901A6A
:101430001968B8EE612AC1F3080101EE901A196823
:10144000F8EE611A40EE201A31EE810A22EE000A0F
:10145000C1F34621491C00EE901AF8EE600A80EEB6
:10146000201AFCEEC10AC0ED000A1968C1F306415A
:10147000491C00EE901AF8EE600A80EE201AFCEE8D
:10148000C10AC0ED010A1968C1F30661491C00EEEA
:10149000901AF8EE600A80EE201ABCEEC10A80EDC8
:1014A000020A30BD074ABFE7284402582C440258BC
:1014B00044440258000000394044025800093D00ED
:1014C0000090D00340787D012DE9F84F0446006874
:1014D00000252E46010104F12400FE4FDFF8F883B9
:1014E00000901DD5606E50B1B0F5801F0CD0B0F5E6
:1014F000001F0ED0B0F5401F1DD001250FE0386849
:1015000040F40030386016E00221201D02F072F82D
:1015100003E00098022102F0E5F805000BD02E460A
:101520002088C00523D5606D05281ED2DFE800F0B5
:101530000C11161B1B00D8F80010626E21F440112C
:101540001143C8F80010EBE7386840F40030386009
:1015500009E00021201D02F04DF803E00098002171
:1015600002F0C0F805466DB100E001252E43208849
:10157000800528D5A06D80281ED00CDC90B14028B5
:101580000ED114E0D8F80010626D21F0070111436C
:10159000C8F80010EBE7C02813D0B0F5807F10D05A
:1015A00001250FE0386840F40030386009E0002180
:1015B000201D02F01FF803E00098002102F092F8CD
:1015C000054685B12E432088DFF8109340052CD5C1
:1015D000D4F8A400B0F5800F20D00DDCA0B1B0F598
:1015E000001F0FD115E0D8F80010A26D21F4E071B2
:1015F0001143C8F80010E6E7B0F5C00F13D0B0F5FE
:10160000000F10D001250FE0386840F4003038603A
:1016100009E00021201D01F0EDFF03E0009800210A
:1016200002F060F8054675B12E43208800052DD5DF
:10163000D4F8A800B0F1007F21D00EDCA8B1B0F141
:10164000807F10D116E0D9F80010D4F8A42021F43E
:1016500060011143C9F80010E7E7B0F1407F13D0F3
:10166000B0F1806F10D001250FE0386840F40030F1
:10167000386009E00021201D01F0BCFF03E0009864
:10168000002102F02FF805466DB12E43206880013D
:101690001FD5A06CD8B110280FD0202812D0302828
:1016A00015D0012514E0D9F80010D4F8A82021F0B5
:1016B000E0611143C9F80010E8E7386840F40030F1
:1016C000386004E00221201D01F094FF05466DB151
:1016D0002E432088C0042BD5E06DB0F5005F20D0EC
:1016E0000DDCA0B1B0F5805F0FD115E07A48001F86
:1016F0000168A26C21F0300111430160E9E7B0F507
:10170000405F13D0B0F5804F10D001250FE038684E
:1017100040F40030386009E00021201D01F06AFF2C
:1017200003E00098002101F0DDFF054685B12E435E
:101730002088800429D5206EB0F5403F23D010DCEE
:1017400008B3B0F5803F14D0B0F5003F0FD115E0DD
:10175000D8F80010E26D21F4E0411143C8F8001000
:10176000E6E7B0F5802F0ED0B0F5A02F0BD0012505
:101770000AE00121201D01F03DFF03E00098012156
:1017800001F0B0FF05468DB12E43208840042AD5D4
:10179000D4F8AC00B0F1405F23D010DC08B3B0F156
:1017A000805F14D0B0F1005F0FD115E0D8F80010C1
:1017B000226E21F4E0211143C8F80010E5E7B0F1F2
:1017C000804F0ED0B0F1A04F0BD001250AE00121CF
:1017D000201D01F00FFF03E00098012101F082FFBE
:1017E00005466DB12E43208800041FD5E06ED8B1A8
:1017F000B0F1805F0ED0B0F1005F10D0012514E091
:10180000D9F80010D4F8AC2021F0E0411143C9F818
:101810000010E8E7386840F40030386004E0012147
:10182000201D01F0E7FE05466DB12E432068C00182
:101830001ED5606CD0B101280ED0022811D003282B
:1018400014D0012513E0D8F80010E26E21F04051C9
:101850001143C8F80010E9E7386840F400303860F8
:1018600004E00221201D01F0C5FE054675B12E439E
:101870002068DFF86CB040025AD51A48016841F47C
:1018800080710160FFF72EFC82460EE01248001FB7
:101890000168626C21F0030111430160E8E7FFF782
:1018A00021FCA0EB0A0064283AD80E480068C00565
:1018B000F5D5B5BB094818300068B4F8B01000F48D
:1018C000407001F44071884219D004481830016812
:1018D0000AE000002C440258504402585844025870
:1018E0001044025800480258026821F4407142F442
:1018F00080320260026822F4803202600160D4F813
:10190000B000B0F5807F22D1FFF7ECFB824609E002
:10191000FFF7E8FBA0EB0A0141F28830814201D9D0
:10192000032504E0FE4800688007F1D57DB12E4311
:101930002078DFF8F0A3C0073CD0A06F182837D07C
:1019400025DC78B3082828D0102824D12BE0D4F83F
:10195000B000C0F3012103290ED0DBF8001021F400
:101960007C51CBF80010EE480168B4F8B020C2F307
:101970000B0211430160DBE7DBF80020EA4B22F4A5
:101980007C5203EA10100243CBF80020EBE720283A
:101990000ED028280CD001250BE00121201D01F0DC
:1019A00029FE04E004E00098012101F09BFE0546B9
:1019B0005DB12E43207880071ED5606F062819D2AE
:1019C000DFE800F0160C11161616DAF80010A26FF8
:1019D00021F038011143CAF80010EBE70121201D66
:1019E00001F008FE03E00098012101F07BFE0546AE
:1019F00075B100E001252E43207840071FD5D4F8AB
:101A00009000062819D2DFE800F0160C1116161601
:101A1000DAF80010626F21F007011143CAF80010D4
:101A2000EAE70121201D01F0E5FD03E00098012116
:101A300001F058FE05469DB100E001252E432078B7
:101A400080062BD5D4F88C00B0F1405F24D011DC97
:101A500010B3B0F1805F15D0B0F1005F10D116E087
:101A6000D9F80010D4F8902021F007011143C9F8EB
:101A70000010E4E7B0F1804F0ED0B0F1A04F0BD0D2
:101A800001250AE00021201D01F0B4FD03E00098CB
:101A9000022101F027FE05468DB12E432078400635
:101AA0002BD5D4F89800B0F5406F24D011DC10B3DA
:101AB000B0F5806F15D0B0F5006F10D116E0DAF8F0
:101AC0000010D4F88C2021F0E0411143CAF8001036
:101AD000E4E7B0F5805F0ED0B0F5A05F0BD0012534
:101AE0000AE00021201D01F085FD03E0009802219D
:101AF00001F0F8FD05468DB12E43207800062BD568
:101B0000D4F89C00B0F5C04F24D011DC10B3B0F570
:101B1000005F15D0B0F5804F10D116E0D9F8001055
:101B2000D4F8982021F4E0511143C9F80010E4E7FB
:101B3000B0F5004F0ED0B0F5204F0BD001250AE0D4
:101B40000021201D01F056FD03E00098022101F064
:101B5000C9FD054665B32E43207800070BD5D4F8A0
:101B60008000B0F5805F2DD0DAF8002022F44052DA
:101B70000243CAF800202078C0060BD5D4F89400A0
:101B8000B0F5807F24D0D9F8002022F440720243BF
:101B9000C9F80020206800032CD5D4F8A000E8B1D3
:101BA000B0F5803F1FD0B0F5003F21D0012520E0E7
:101BB000D9F80010D4F89C2021F460411143C9F8F1
:101BC0000010C9E70098022101F08CFD0643D2E71E
:101BD0000098022101F086FD0643DBE70021201D6D
:101BE00001F008FD03E00098022101F07BFD0546AD
:101BF00085B12E432068400322D5D4F88400B0F587
:101C0000801F11D0B0F5001F13D0B0F5401F15D0C4
:101C1000012514E0D9F80010D4F8A02021F44031B7
:101C20001143C9F80010E5E7386840F40030386027
:101C300004E00098012101F055FD054655B12E4301
:101C40002068C0031CD5E06C70B1B0F5803F10D0A7
:101C5000012514E0DAF80010D4F8842021F44011B2
:101C60001143CAF80010EBE7386840F400303860E0
:101C700004E00221201D01F0BDFC0546C5B12E4344
:101C80002068800004D50098022101F02BFD064356
:101C9000206880031BD5E06FB8B1B0F5807F10D00D
:101CA000B0F5007F11D0B0F5407F0ED001250DE0DA
:101CB0001C4808380168E26C21F48031114301604E
:101CC000DEE7386840F40030386045B32E432068C2
:101CD000C00207D5D8F80000226F20F00040104362
:101CE000C8F800002068C00008D5DBF80010D4F860
:101CF000B42021F480411143CBF800102068800209
:101D000007D5D8F80010A26E21F080711143C8F8F1
:101D100000102068400014D5DBF8001006E01EE03B
:101D20007044025854440258CFFFFF0021F4004190
:101D3000CBF80010DBF80010D4F8B8201143CBF832
:101D400000102068002806DA0A480168226D21F098
:101D50004051114301605EB10120BDE8F88FDAF80F
:101D60000010E26F21F440711143CAF80010AEE791
:101D70000020F2E74C4402582DE9F047DFF8BC910F
:101D800004460E46D9F8000000F00700B0420CD21D
:101D9000D9F8001021F007013143C9F80010D9F833
:101DA000000000F00700B0427ED12078DFF890817B
:101DB000800707D5D8F80010E26821F00F01114321
:101DC000C8F800102078C00762D0D8F80010A268C8
:101DD00021F470611143C8F800105949606818393E
:101DE00002281CD003281DD0096801281DD04907EE
:101DF000002960DA524F083F396821F0070101439A
:101E00003960FFF76FF90546606841F288310228B2
:101E100013D003281ED001288A4627D034E0096851
:101E20008903E5E709688901E2E7C905E0E7FFF70B
:101E300059F9411B514501D923E08A463868C0F35E
:101E4000C2000228F3D123E0FFF74CF9411B5145B2
:101E500001D916E08A463868C0F3C2000328F3D1DE
:101E600016E0FFF73FF9411B51450AD83868C0F327
:101E7000C2000128F5D10BE0FFF734F9411B5145B1
:101E800002D90320BDE8F087386810F0380FF3D18D
:101E9000D9F80010484601F00701B1420DD9016898
:101EA00021F00701314300E005E00160006800F027
:101EB0000700B04201D00120E4E72078400707D5B1
:101EC000D8F80010226921F070011143C8F8001001
:101ED000207801071B4805D50168626921F070016F
:101EE000114301602178C90605D50168A26921F472
:101EF000E061114301602078800607D51149091D72
:101F00000868E26920F070001043086000F066F88D
:101F1000D8F800104FF4807292FAA2F201F47061C6
:101F2000B2FA82F2D140084A515CC84007490860C1
:101F30000F20FFF7F3F80020A4E700000020005274
:101F4000184402581C440258E54700080C000024BD
:101F500010B5FFF78DF908490968012292FAA2F23B
:101F600001F00F01B2FA82F2D140044A515CC8403C
:101F70000349086010BD000018440258E5470008F6
:101F80001000002410B5FFF7E3FF0749096810228D
:101F900092FAA2F201F07001B2FA82F2D140034A41
:101FA000515CC84010BD00001C440258E5470008C1
:101FB00010B5FFF7CDFF074909684FF4807292FA18
:101FC000A2F201F4E061B2FA82F2D140024A515C1D
:101FD000C84010BD1C440258E54700083548F0B51C
:101FE0000068364D10F03801334809D00411082933
:101FF00004D0334E10290BD018290BD02046F0BD49
:1020000029688906FBD52968C1F3C101C840F0BD24
:102010003046F0BD274918310A68096812F00302FA
:10202000284BC1F305111B68274F03F001033F68DC
:10203000DFED260AB7EE001AC7F3CC0717FB03F350
:1020400000EE103A224BB8EE400A06D0012A01D029
:10205000022A2BD0B4FBF1F008E02A68920603D5DF
:102060002A68C2F3C102D040B0FBF1F001EE900A41
:102070001868B8EE612AC0F3080001EE900A1868EB
:10208000F8EE611A40EE201A31EE810A22EE000AC3
:10209000C0F34620401C00EE900AF8EE600A80EE85
:1020A000201ABCEEC10A10EE100AF0BDB6FBF1F02A
:1020B000DCE70000104402580090D00300440258AE
:1020C00040787D012C440258344402580000003905
:1020D000304402582DE9F05F04460078DFF8FC83B5
:1020E00041F28839DFF8F8A3FE4DC0074ED0D8F88A
:1020F00000104046C1F3C20102291AD00068C0F3A3
:10210000C200032805D1DAF8000000F0030002281D
:102110000FD06068B0F5803F12D010B1B0F5A02F9D
:1021200019D0286820F480302860286820F48020A6
:1021300009E02868800329D56068002874D025E06C
:10214000286840F480302860606890B1FEF7CAFFCC
:1021500006464F4609E0286840F480202860EFE7F3
:10216000FEF7C0FF801BB8427DD828688003F7D5F2
:102170000CE0FEF7B7FF06464F4604E0FEF7B2FF5D
:10218000801BB842F0D828688003F7D42078D64F57
:1021900080075AD5D8F8001040464FF47C3B11F028
:1021A000380F13D00068C0F3C200032803D1DAF857
:1021B000000080070AD0E068A8B3296821F019015F
:1021C00001432960FEF78EFF06461DE028684007A0
:1021D00002D5E0680028B1D02868E16820F0190035
:1021E00008432860FEF77EFF064604E0FEF77AFF0C
:1021F000801B0228B8D828684007F7D507E0FEF70B
:1022000071FF801B0228AFD828684007F7D53868CF
:102210009BFAABF220F47C312069B2FA82F2904052
:102220000143396011E000E0AEE0286820F00100D1
:102230002860FEF757FF064604E0FEF753FF801BB9
:10224000022891D828684007F7D42078C00655D5D1
:10225000D8F8001040464FF0F84BC1F3C2010129F5
:1022600017D0006800E0EDE0C0F3C200032805D1FC
:10227000DAF8000000F0030001280AD0E069002825
:1022800028682CD040F080002860FEF72BFF06461F
:1022900016E02868C00502D5E069802874D1386846
:1022A0009BFAABF220F0F841206AB2FA82F2904039
:1022B0000143396022E0FEF715FF801B022899D800
:1022C0002868C005F7D538689BFAABF2216AB2FAE4
:1022D00082F220F0F8409140084338600EE020F090
:1022E00080002860FEF7FEFE064604E0FEF7FAFED8
:1022F000801B022887D82868C005F7D420780007FB
:1023000024D5774F60694C37002838680FD040F0EB
:1023100001003860FEF7E6FE064604E0FEF7E2FE46
:10232000801B02288DD838688007F7D50EE020F092
:1023300001003860FEF7D6FE064604E0FEF7D2FE46
:10234000801B02287ED838688007F7D42078800662
:1023500023D5A069002828680FD040F48050286059
:10236000FEF7C0FE064604E0FEF7BCFE801B022816
:1023700068D828688004F7D50FE020F480502860E2
:10238000FEF7B0FE064605E0D6E0FEF7ABFE801B8A
:10239000022857D828688004F7D42078400744D50D
:1023A000524F386840F480703860FEF79BFE064656
:1023B00004E0FEF797FE801B642843D83868C00508
:1023C000F7D5474FA068483701280AD008B105283B
:1023D00011D0386820F001003860386820F004001F
:1023E00002E0386840F001003860A06888B1FEF76C
:1023F00079FE064609E0386840F004003860F0E7EE
:10240000FEF770FE811B49451CD838688007F7D558
:102410000BE0FEF767FE064604E0FEF763FE811B55
:1024200049450FD838688007F7D4606AF0B3D8F808
:102430000010C1F3C20103297ED00228286820F0D1
:10244000807000E079E0286003D0FEF74BFE044680
:1024500087E0FEF747FE064604E0FEF743FE801BDA
:1024600002287BD828688001F7D4DAF8001040F2FF
:10247000F3329143E26A41EA0211A26A1143CAF8B7
:10248000001094F834004FF4FE02218E4002491EE1
:10249000A0F5007080B2C1F308010843218F491EE6
:1024A00002EA0141084394F83C1000E05CE0491E58
:1024B000120202EA016108430949083108600B1D54
:1024C00019684FF6F872A06C914392FAA2F2B2FA30
:1024D00082F2904001431960014809E0104402581B
:1024E0002844025800440258044402580048025844
:1024F000001D0168226C21F00C011143016001688C
:10250000626C21F0020111430160016841F48031E5
:102510000160016841F400310160016841F48021EB
:102520000160016841F001010160286840F080709D
:102530002860FEF7D7FD01E018E00FE0044604E054
:10254000FEF7D0FD001B022808D828688001F7D5C7
:102550000AE0FEF7C7FD001B022802D90320BDE8F0
:10256000F09F28688001F4D40020F8E70120F6E706
:102570002DE9F05F04004FF000053DD0DFF8C48185
:102580002068714E714F4045A36A06D0B04204D016
:10259000B84202D0E1680F292ED8E26B4FF0010B50
:1025A0000BEB521CE26802F10801C908404501FB2F
:1025B0000CF105D0B04203D0B84201D008291BD895
:1025C000404503D0B04201D0B84201D1102913D800
:1025D0004FF480094B4512D1404507D0B04205D099
:1025E000B84203D0206BB0F5702F05D8256B05B924
:1025F0001504B2EB154F02D90120BDE8F09F94F805
:1026000081004FF0000A20B9204684F880A000F035
:102610009FF8022084F881002068016821F0010100
:102620000160A069B0F1806F09D16068484506D1AA
:10263000A06B20B92068016841F480510160A16A53
:10264000E0690843E16B29430843E16808432168D6
:102650008860616A606BA2690843A16B11430843FB
:102660002169084361690843216A08436168084396
:10267000E16C0843A1680843A16C0843A16D0843BD
:102680002168C860A06A484529D1206C01282068CB
:10269000016827D021F400410160606C01282068A6
:1026A000016822D021F4804101602068404506D0B5
:1026B000B04204D0B84202D0B5F5702F18D04045D2
:1026C00003D0B04201D0B84202D1B5F5F81F0FD007
:1026D000016821F4005101602168E06A08646068C3
:1026E00050B119E041F40041D6E741F48041DBE705
:1026F000016841F40051EEE7A06A30B920688168B2
:1027000021F4C05141F4006181602068816821F4A6
:10271000C06141F4806181602068016D21F0010198
:1027200001656068400206D52068C168626D21F0CD
:1027300000411143C160C4F884A084F881B0002036
:102740005BE700000030014000380040003C0040E2
:10275000164800B5B5B0016841F00201016000689B
:1027600000F00200349011480830016841F48041C3
:102770000160006800F4804034904FF48050009075
:10278000002017906846FEF79FFE4FF460402F90A0
:1027900002203090012031900320329005203390A8
:1027A00003482FA9FEF79CFB35B000BDE04402585A
:1027B000000402582DE9F84F044690F880001F46A7
:1027C00092460A9D01288B4613D04FF0010984F8E8
:1027D0008090FEF787FC94F8812006460020012AAD
:1027E0004FF480010ED062688A4209D1A2683AB9DA
:1027F00002E00220BDE8F88F94F88120042A01D07D
:10280000022136E0BBF1000F32D0BAF1000F2FD019
:1028100077B394F88120042A02D0052284F881201D
:102820008046C4F88400C4F864A0A4F86A70A4F8D0
:102830006870C4F85CB0A4F86270A4F86070206797
:102840006067206842686FF30F023A434260206875
:10285000026842F0010202606068884204D1206888
:10286000016841F400710160E0680F2840D848E039
:10287000012184F880000846BCE7B4F8620070B11A
:102880002068416989070AD5E16D09680162E06D38
:10289000001DE065B4F86200401EA4F86200B4F8C0
:1028A0006A0080B12068416948F2080211420AD0EA
:1028B000006B616E0860606E001D6066B4F86A00AF
:1028C000401EA4F86A00681C12D0FEF70BFC801BA7
:1028D000A8420DD3204600F0D3FF84F88080D4F8BE
:1028E000840040F48070C4F8840084F88190EBE0A8
:1028F000B4F862000028C0D1B4F86A000028BCD146
:10290000C8E0072849D8BDE0B4F86200F0B12068FB
:10291000416989071AD5B4F8621001290BD9E16B16
:1029200049B1E16D09680162E06D001DE065B4F830
:102930006200801E08E0E16D09880184E06D801C62
:10294000E065B4F86200401EA4F86200B4F86A00C2
:10295000E0B12068416911F4604F17D04169090462
:1029600009D5006B616E0860606E001D6066B4F88A
:102970006A00801E08E0008E616E0880606E801C18
:102980006066B4F86A00401EA4F86A00681C04D0AF
:10299000FEF7A8FB801BA8429CD2B4F86200002876
:1029A000B2D1B4F86A000028AED173E0B4F8620086
:1029B00080B32068416989072CD5B4F862100329D7
:1029C0000CD9E16B402909D9E16D09680162E06D1C
:1029D000001DE065B4F86200001F19E0B4F8621051
:1029E00001290BD9E16B49B1E16D09880184E06DE2
:1029F000801CE065B4F86200801E09E0E16D097892
:102A000080F82010E06D401CE065B4F86200401EC4
:102A1000A4F86200B4F86A0068B32068416911F450
:102A2000604F28D04169090409D5006B616E0860C8
:102A3000606E001D6066B4F86A00001F19E041690D
:102A400001F4C041B1F5005F09D9008E616E0880C4
:102A5000606E801C6066B4F86A00801E09E090F821
:102A60003000616E0870606E401C6066B4F86A00E9
:102A7000401EA4F86A00681C04D0FEF733FB801BDC
:102A8000A84289D2B4F8620000288FD1B4F86A0055
:102A900000288BD10022334608212046009500F003
:102AA0005EFF28B1D4F8840040F02000C4F8840010
:102AB000204600F0E5FE84F8808084F88190D4F808
:102AC000840000283FF4D8AE012093E64FF0E021C7
:102AD0000428086903D020F004000861704740F022
:102AE0000400FAE7401EB0F1807F10B501D3012049
:102AF00010BD4FF0E02460610F21601701F00BFD65
:102B00000020A06107202061002010BD70477047A1
:102B100090F8791090F87A000843704770B5026811
:102B20000446D0691368916810F00F0F64D0594DB6
:102B300003F490760D40354376D0C50707D0DD0508
:102B400005D501251562E26F42F00102E2678207B6
:102B500008D5CA0706D0256802222A62E26F42F031
:102B60000402E267420708D5CA0706D02568042296
:102B70002A62E26F42F00202E26702070ED503F01A
:102B8000200201F080552A4352EAC17206D025681E
:102B900008222A62E26F42F00802E267E26F002A2E
:102BA0003AD0800608D503F0200001F08051084398
:102BB00002D0204601F090F9E06F000703D42068AE
:102BC000806840062AD5204601F078F9206881689F
:102BD00049061ED5816821F040018160606FC0B157
:102BE0002D490165606FFEF719F8002814D0606F59
:102BF000016DBDE870400847850615D503F0200536
:102C000001F0805635430FD02046BDE8704001F0FA
:102C100063B92046FFF77BFF70BD05E02046FFF754
:102C200076FF0020E067F7E7C6024FF020050CD5DD
:102C30004E020AD5E803106284F8795084F87A507D
:102C40002046BDE87040FFF761BF06060AD503F0D5
:102C5000800601F400010E4304D02046BDE8704018
:102C600001F0CABB41060BD5590609D511682046AB
:102C700021F04001116084F8795000F005F9CBE7AC
:102C80000002C9D55800C7D5106820F080401060F8
:102C9000C2E7000001000010A93E000810B50400C2
:102CA00003D094F8790010B107E0012010BD002096
:102CB00084F87800204600F027F8242084F8790072
:102CC0002068016821F001010160204601F040F90F
:102CD0000128EBD0606B10B1204601F053F820685A
:102CE000416821F4904141602068816821F02A0107
:102CF00081602068016841F0010101602046BDE863
:102D0000104001F0A3B8000010B5006886B01B4960
:102D1000884230D11A48016841F001010160006821
:102D200000F00100059016481030016841F01001D4
:102D3000016000680121134C00F0100005904FF471
:102D4000007000900220CDE9010103900720694640
:102D500004902046FEF7C4F84FF4806120460091AD
:102D60006946FEF7BDF82520FEF743FA0322252029
:102D70001146FEF74BFA06B010BD000000100140EE
:102D8000E04402580000025890F87A30202B4CD1D1
:102D9000B9B1B2B190F87830012B46D0012380F858
:102DA00078304166A0F86820A0F86A20FF22816888
:102DB000B1F5805F07D07F2351B1B1F1805F0CD0B6
:102DC00010E001207047016921B940F2FF1107E0CE
:102DD000016909BBA0F86C2004E00169E1B13F2161
:102DE000A0F86C100021C167222280F87A2080F8B8
:102DF000781001688A6842F001028A6001680A68F6
:102E000092000CD50A6842F480720A6000688168FA
:102E100041F08051816006E0A0F86C30E2E708687C
:102E200040F4907008600020704702207047000056
:102E300030B50068114988420CD1114A508801040C
:102E400008D411464FF000034404097806D50A2936
:102E500001D0538030BD40F400400DE00D2909D071
:102E6000084DC0F30D04401C80B2C728295550807E
:102E7000EFD830BD40F48040508030BD001001409C
:102E800018000024300000247047FEE7144870B595
:102E900086B0016841F004010160016801F004019D
:102EA0000591016841F010010160006800260325CA
:102EB000694600F01000059008200124CDE90006C5
:102EC0000848CDE90245FEF70BF820206946CDE918
:102ED00000060548CDE90245FEF702F806B070BDD0
:102EE000E044025800100258000802582DE9F04151
:102EF0001C4C01251C4E01281C4F12D0207848B1D3
:102F000008213046FEF7E0F868B120213846FEF788
:102F1000DBF840B108213046FEF7D6F8012817D07B
:102F20001DE02570ECE70A2001F01EFB0020207058
:102F300008213046FEF7C8F828B120213846FEF7B0
:102F4000C3F818B10BE00120BDE8F0810220FBE7D7
:102F500020213846FEF7B8F8012800D1257000205E
:102F6000F2E7000028000024001002580008025870
:102F70002DE9F0410D4F00240646214620467B886E
:102F80003A8800F0E1F93D880021788845430846F9
:102F900000F0C6F900F0C0FA03E0304600F066FA2F
:102FA000641CAC42F9D3BDE8F08100001C0200248F
:102FB0002DE9F0411E490027F0222C242A252B263A
:102FC0004FF4A07338B1012817D002284FF0010C3C
:102FD0001BD0032822D08F710A804B800C810024E3
:102FE0004D818E814B880A880021084600F0ACF99B
:102FF0002046BDE8F04100F081B98F710B804A8016
:103000000C8101244D818E81ECE781F806C00A8095
:103010004B800C8102244D818E81E3E781F806C04C
:103020000B804A800C8103244D818E81DAE70000F9
:103030001C0200242DE9F0410B4C16460F460546B4
:10304000608900F04DFA284600F010FAA08900F0DF
:1030500047FA384600F00AFA208900F041FA304673
:10306000BDE8F04100F002BA1C0200242DE9F04155
:103070005C1A151A641C069F6D1CA3B2AAB200F05C
:1030800063F90B4E308900F02BFA654300F044FAE7
:10309000002403E0384600F0E9F9641CAC42F9D999
:1030A0007388002132880846BDE8F04100F04CB931
:1030B0001C0200241A4810B586B0016841F00201D4
:1030C000016000686946174C00F00200059041F26B
:1030D00003000090012001900290032003902046FD
:1030E000FDF7FEFE012220461146FDF7F6FF012204
:1030F00020460221FDF7F1FF012220461103FDF7D2
:10310000ECFF00F067FBA00400F0A2FB00F00CF85D
:10311000012220461146FDF7E0FF06B010BD000079
:10312000E04402580004025870B50A4D4FF4804440
:10313000002221462846FDF7D0FF322001F014FA84
:10314000012221462846FDF7C8FFBDE870401E2039
:1031500001F00ABA0004025810B5FFF7ABFF00F007
:103160007BF9322001F000FA362000F0B9F9002096
:1031700000F09AF93A2000F0B3F9052000F094F934
:10318000B22000F0ADF90C2000F08EF90C2000F018
:103190008BF9002000F088F9332000F085F9332006
:1031A00000F082F9B72000F09BF9352000F07CF99F
:1031B000BB2000F095F9192000F076F9C02000F04E
:1031C0008FF92C2000F070F9C22000F089F901205D
:1031D00000F06AF9C32000F083F9122000F064F9CE
:1031E000C42000F07DF9202000F05EF9C62000F038
:1031F00077F90F2000F058F9D02000F071F9A420E1
:1032000000F052F9A12000F04FF9E02000F068F939
:10321000D02000F049F9042000F046F90D2000F01C
:1032200043F9112000F040F9132000F03DF92B2064
:1032300000F03AF93F2000F037F9542000F034F95B
:103240004C2000F031F9182000F02EF90D2000F08C
:103250002BF90B2000F028F91F2000F025F923207E
:1032600000F022F9E12000F03BF9D02000F01CF939
:10327000042000F019F90C2000F016F9112000F0DC
:1032800013F9132000F010F92C2000F00DF93F2065
:1032900000F00AF9442000F007F9512000F004F989
:1032A0002F2000F001F91F2000F0FEF81F2000F091
:1032B000FBF8202000F0F8F8232000F0F5F821209A
:1032C00000F00EF9112000F00BF9782001F04CF914
:1032D000292000F005F9C82001F046F90020FFF789
:1032E00067FE012204481146FDF7F7FEBDE81040D5
:1032F0004FF6FF70FFF73CBE00040258002158B1A2
:10330000012804D0022804D0032805D103E060215D
:1033100002E0C02100E0A021362000F003B9000047
:1033200070B5084C0D460646608900F0D9F8304665
:1033300000F09CF8A08900F0D3F82846BDE8704062
:1033400000F094B81C0200242DE9F04104460E4F11
:1033500010448846401E86B2C818401E85B278893F
:1033600000F0BEF8204600F081F8304600F07EF80C
:10337000B88900F0B5F8404600F078F82846BDE876
:10338000F04100F073B800001C0200242DE9F84F52
:103390001F460C4682468B46580700D0012079080C
:1033A00000EBD700203A10FB01F0002602F0FF09E5
:1033B000C0B2009040E00C2F0FD0102F11D0182F6A
:1033C0003DD1204909EBC90001EB80004FF0000816
:1033D000855D280609D50A9A0BE01B4909EB4900CF
:1033E000F2E71A4901EB0910F0E70B9828B91848E1
:1033F000428821465046FFF71DFE6806641C050EF4
:103400001448A4B24088A04219D9A4EB0B00B842DA
:1034100009D10AF101005C461FFA80FA0D480188C3
:1034200051450CD906E008F1010000F0FF08B8F1A1
:10343000080FCED3761CF6B200988642BBD3BDE807
:10344000F88F0000725200080E480008824C0008F5
:103450002A0000241C020024012010B500F040F8CE
:10346000BDE81040322001F07FB8000070B50D4E6D
:103470004FF480550022044629463046FDF72DFEC4
:10348000012230460221FDF728FE200A00F0D0F983
:10349000E0B200F0CDF929463046BDE87040012287
:1034A000FDF71BBE0004025870B50C4D4FF480545C
:1034B0000022064621462846FDF70FFE0122284637
:1034C0000221FDF70AFE304600F0B2F921462846F7
:1034D000BDE870400122FDF700BE00000004025864
:1034E00070B50C4E4FF480550022044629463046F4
:1034F000FDF7F3FD002230460221FDF7EEFDE0B2BC
:1035000000F096F929463046BDE870400122FDF7EB
:10351000E4BD00000004025801480089FFF7E0BF45
:103520001C02002410B50C46FFF7DAFFE0B2BDE83C
:103530001040FFF7B9BF00000E4810B586B0016813
:1035400041F001010160006869460B4C00F0010088
:10355000059002200090012001900290032003902A
:103560002046FDF7BDFC012220460221FDF7B5FDF6
:1035700006B010BDE0440258000002580EB500210C
:10358000012000900323CDE90101122102464806E3
:1035900000F001F80EBD2DE9FF4707461E460CA8B6
:1035A00014460D4690E80007FDF702FE01208DF855
:1035B000000000208DF808508DF80C008DF80900EF
:1035C0008DF80D808DF80A0068468DF80E908DF804
:1035D000014001978DF80B608DF80FA0FDF7BEFD3F
:1035E0000420FDF7F3FD04B00020BDE8F08770472C
:1035F000704700002DE9F047DFF8E48004460F46ED
:103600004FF00009D8F80000C043800709D0344DBE
:10361000283D286820F080602860FDF763FD06469D
:1036200007E00120BDE8F087FDF75CFD801B022864
:103630004ED828680001F7D4D8F80010226821F489
:103640007C3141EA0231C8F80010207A4FF4FE02C2
:10365000A1884002491EA0F5007080B2C1F30801A4
:103660000843A189491E02EA01410843217C120254
:10367000491E02EA016108431949103108601848DF
:10368000001D0168626921F0C001114301600168F9
:10369000A26921F02001114301606FB10168012F7F
:1036A0000ED041F400110160286840F0806028606D
:1036B000FDF718FD04460DE0016841F40021F2E732
:1036C00041F48011EFE7FDF70DFD001B022801D941
:1036D0000320A7E728680001F5D54846A2E70000C7
:1036E000284402582DE9F047DFF8E48004460F46ED
:1036F0004FF00009D8F80000C043800709D0344DCE
:10370000283D286820F080502860FDF7EBFC064635
:1037100007E00120BDE8F087FDF7E4FC801B0228EC
:103720004ED828688000F7D4D8F80010228821F0FD
:103730007C7141EA0251C8F80010207A4FF4FE0271
:10374000A1884002491EA0F5007080B2C1F30801B3
:103750000843A189491E02EA01410843217C120263
:10376000491E02EA016108431949183108601848E6
:10377000001D0168626921F4406111430160016824
:10378000A26921F40071114301606FB10168012F3A
:103790000ED041F080710160286840F080502860B0
:1037A000FDF7A0FC04460DE0016841F48001F2E75A
:1037B00041F40001EFE7FDF795FC001B022801D959
:1037C0000320A7E728688000F5D54846A2E7000057
:1037D0002844025810B5154C072113484FF00072C9
:1037E00004F1080320604FF480006060002083E84B
:1037F0000700521062619200A261CA0760636265AD
:103800000A07C4E907206062C4E90A012046FEF7FE
:10381000AFFE2068016841F001010160BDE8104081
:10382000FF2000F005B8000000380040940100249B
:1038300001B582B04FF47A700123009001AA0348C9
:1038400002A9FEF7B7FF9DF804000EBD9401002405
:103850000A4A11680B6823F001030B6011688B683A
:1038600023F0E0438B6011688B6803438B60106822
:10387000016841F0010101607047000094010024DB
:1038800010B502685169936943F0080393610268B7
:10389000936943F0100393610268136823F00103F6
:1038A00013600268136940F26B34A343136102682A
:1038B000936823F44043936090F88120042A0CD04D
:1038C0008A060AD5D0F8842042F08002C0F884200D
:1038D0000268936943F02003936190F88120032AE2
:1038E0001DD04A060AD5D0F8842042F00402C0F860
:1038F00084200268936943F040039361826AB2F5C1
:10390000800F0CD10A060AD5D0F8842042F00202BA
:10391000C0F884200268936943F0800393618A05AC
:103920000AD5D0F8842042F00102C0F88420026851
:10393000936943F400739361C9050AD5D0F88410E4
:1039400041F00801C0F8841001688A6942F480726D
:103950008A610021A0F86210A0F86A1010BD2DE95C
:10396000F0411E4617460D468046069C0AE0601C44
:1039700008D024B1FDF7B6FB801BA04202D903207A
:10398000BDE8F081D8F80000406935EA000004D0B5
:103990000020B842EBD00020F2E70120F9E7000058
:1039A0001249884201D2002070471149884201D251
:1039B000012070470F49884201D2022070470E490A
:1039C000884201D2032070470C49884201D204206A
:1039D00070470B49884201D2052070470949884247
:1039E00001D206207047072070470000000002083F
:1039F00000000408000006080000080800000A088B
:103A000000000C0800000E08002310B503E010C8E9
:103A100041F823405B1C9342F9D310BD2DE9F04FD0
:103A200087B01746B0F1006F0E4604464FF0000A0B
:103A3000CDF814A059D3A00757D1FDF737FA2C4879
:103A400004EB870725464CF2503B844238D339E0DB
:103A50002868401C2FD0D0462846CDF800A0FFF79C
:103A60009FFF02900120019005A90390202004905F
:103A70006846FDF725F928BB1E49C1F80080BFF351
:103A80004F8F081F006843F6FF79DFF86C80C0F3A2
:103A90004E31C0F3C90C09EA4113604643EA807213
:103AA000C8F80020401EF9D2491EF4D2BFF34F8F50
:103AB000BFF36F8F00E02D1D58460121FCF738FE43
:103AC000BD42C5D301215846FCF732FE48B10AE099
:103AD0000023324603202146FDF782F918B920342D
:103AE0002036BC42F4D3FDF76BF907B0BDE8F08F88
:103AF0000000F01F84ED00E074EF00E0704700006C
:103B00002DE9F04F93B01F4615468A46044681467C
:103B1000580700D0012000EBD7000C2F10FB07F056
:103B2000C0B2129003D0102F01D0182F2FD102460F
:103B300069462846FDF748F8002024E01DF8086093
:103B40000025DFF850B0300601D51C9A03E01D981F
:103B500028B9BBF8002051462046FFF76BFA7006E3
:103B6000641CA4B2060EA4EB0900B84204D10AF109
:103B700001004C461FFA80FA6D1CEDB2082DE2D30D
:103B800008F10100C0B2129980468842D6D313B022
:103B9000BDE8F08F2C0000242DE9FF4F83B09B4639
:103BA0000E46044680468A46DDE9107500208146AF
:103BB0001FE0B9F1000F22D005994FF0000908EB82
:103BC0000100401BA04202DA7019444686B20AEB9B
:103BD0000B00401BB0420FDBDDE912012B463A46D9
:103BE000CDE9000131462046FFF78AFF601984B213
:103BF000BF1C3A78002ADCD107B0BDE8F08F802ADC
:103C000001D90120D3E7059908EB0100A0EB55008D
:103C1000A04202DA7019444686B20AEB0B00401B40
:103C2000B042E9DB0D2A0DD0DDE912012B46CDE9CA
:103C3000000131462046FFF7A9FB04EB550084B292
:103C40007F1CD6E77019444686B27F1CF5E700005A
:103C500070B5284C9CB0256825F004052560254CDE
:103C600000260C34256845F440452560256805F498
:103C700040451B952568AD04FCD5012400940CAD8E
:103C800003962404019402240994CDE90A4107967D
:103C9000082485E80D00CDE910466846FEF71AFABB
:103CA00088B93F2013900320CDE91406402001017C
:103CB000CDE91640CDE9180150201A90022113A831
:103CC000FEF75AF810B101201CB070BD0A48016817
:103CD00041F0800101600848F430016841F00201C0
:103CE0000160006800F002001B90FCF7E1FF00207B
:103CF000EAE700000C48025800440258FDF7F8B902
:103D00001C48016841F4700101601B49086840F0DB
:103D100001000860184A0020103210600A68174B32
:103D20001A400A60144A18321060121D1060121DE9
:103D30001060114A28321060121D1060121D1060B0
:103D4000121D1060121D1060121D1060121D1060F7
:103D5000121D10600A6822F480220A600649603150
:103D6000086001200649C1F80801C00601498039F0
:103D70000860704788ED00E0004402587FEDF6EAE5
:103D80000080005190F83410C90706D001684A68D5
:103D9000836B22F400321A434A6090F8341089078A
:103DA00006D501684A68C36B22F480321A434A6020
:103DB00090F83410490706D501684A68036C22F46C
:103DC00080221A434A6090F83410090706D501682A
:103DD0004A68436C22F400421A434A6090F8341057
:103DE000C90606D501688A68836C22F480521A439A
:103DF0008A6090F83410890606D501688A68C36C19
:103E000022F400521A438A6090F83410490611D502
:103E100001684A68036D22F480121A434A60016DFA
:103E2000B1F5801F06D101684A68436D22F4C002D3
:103E30001A434A6090F83410090606D501684A68AA
:103E4000806D22F4002202434A607047F8B50025D5
:103E50000446C567FDF746F90746206800686FF01D
:103E60007E46000708D500223B464FF4001120464D
:103E7000009600F0FBFA60B92068006840070AD598
:103E800000223B464FF480012046009600F0EEFAF7
:103E900008B10320F8BD202084F8790084F87A0066
:103EA000002084F87850F8BD10B5806B0021A0F890
:103EB0006A10A0F86210FEF72AFE10BD01680A68B9
:103EC00022F490720A6001688A6822F001028A6016
:103ED000202180F87A10704710B5B0F86C2090F867
:103EE0007A300168222B05D0088B40F00800088347
:103EF000022010BD898C8368B3F5805F01D103690E
:103F00006BB11140426E531C43661170B0F86A10D9
:103F1000491E0904090CA0F86A1007D015E0436E89
:103F200011401980416E891C4166EFE701680A68FB
:103F300022F490720A6001688A6822F001028A60A5
:103F4000202180F87A10FEF773FF002010BD0000DA
:103F50002DE9F04F044600688025FD4B0021D4F880
:103F600010C087B0A6680F46D4F81C8046EA0C063D
:103F7000D4F814C0A26A4CEA080C46EA0C06324394
:103F80000668DFF8D0C306EA0C0616430660206810
:103F90004268E66822F44052324342602268A069D7
:103FA0009A4201D0266A3043A66AB6F1005F04D176
:103FB000D4E90B6C46EA0C0630439668DFF898C3E8
:103FC00006EA0C06064396602068C26A666A22F01A
:103FD0000F023243C262E14E2068E14AB04210D182
:103FE000126802F03802182A74D005DCCAB3082A15
:103FF0007AD0102A47D179E0202A7BD0282A7CD198
:104000007AE0D84EB04209D1126802F00702062ABF
:1040100073D2DFE802F053696B6D6F71D24EB0421C
:1040200009D1126802F00702062A66D2DFE802F020
:10403000465C5E606264CD4EB04209D1126802F007
:104040000702062A59D2DFE802F0394F515355577B
:10405000C74EB0420BD1126802F00702062A4CD2BA
:1040600000E00EE0DFE802F02A4042444648C14E3C
:10407000B04209D1126802F03802182A38D0BBDCED
:10408000B4E74FF0010538E0BB4EB04209D11268E9
:1040900002F00702062A30D2DFE802F01026282AB2
:1040A0002C2EB64EB0420BD1126802F00702062A3F
:1040B00023D2DFE802F003191B1D1F2100251CE09D
:1040C00098421AD1A64A121D126802F00702062A67
:1040D00013D202E00CE007E00CE0DFE802F0030599
:1040E00007090B0D022508E0042506E0402504E041
:1040F000082502E0102500E02025DFF864B2A04E7C
:104100009842DFF880A2ABF1540B73D1102D31D05F
:1041100006DC022D09D0042D0AD0082D2FD111E084
:10412000202D29D0402D2AD107E0FDF7BBF813E060
:104130006846FDF7CDF801980EE003A8FDF746F9B3
:10414000049809E0DBF800105846890610D500688D
:10415000C0F3C1012AFA01F0002811D06168894634
:1041600001EB410181420AD8B0EB093F07D808E0D2
:104170005046F3E78448F1E74FF40040EEE70127AB
:1041800033E1102D4FF000084ED006DC022D0FD089
:10419000042D15D0082D04D12DE0202D4AD0402D1E
:1041A00013D00127794AA0F54071914270D9E6E712
:1041B000FDF778F8626A0023414636F812200DE0D8
:1041C0006846FDF785F8019803E003A8FDF7FEF8BF
:1041D00004980023616A36F811201946FCF778F834
:1041E00062680902030241EA10615008181841EBA5
:1041F000080115E032E0DBF800105846890609D5C1
:1042000000680023C0F3C1012AFA01F0616A36F8A0
:10421000112015E0606A002336F8102050460FE0A8
:104220000023FCF755F8BDE7606A002336F810203C
:10423000554805E0606A002336F810204FF400402E
:104240000021FCF745F80902020241EA10614FEA39
:10425000590010184A4641EB0801E1E7E3694FF4C1
:10426000004293424DD1082D23D005DC8DB1012DA4
:1042700012D0042D06D112E0102D35D0202D3AD0C9
:10428000402D11D0012721F00F00C1F34201084356
:104290005AE0FDF777FE16E0FDF78AFE13E0684668
:1042A000FDF716F801980EE003A8FDF78FF80498C3
:1042B00009E0DBF800105846890608D50068C0F30D
:1042C000C1012AFA01F0616A36F8111010E0606A43
:1042D00036F81010BAFBF1F04100606801EB5001B4
:1042E000B1FBF0F081B2CEE7606A36F810102648D4
:1042F000B0FBF1F0F0E7606A36F81000B2FBF0F0C6
:10430000EAE7082D4AD00ADC0DB3012D43D0042D75
:104310007FF44DAF6846FCF7DBFF019809E0102DF4
:1043200052D0202D55D0402DF2D103A8FDF74EF8E4
:104330000498616A36F81110B0FBF1F1606801EB86
:104340005001B1FBF0F080B22168C8604DE01FE081
:10435000000C0058F369FFCFFFF4FF11001001407B
:10436000544402580044004000480040004C0040C3
:10437000005000400014014000780040007C0040E4
:10438000F64700080090D00300093D00FFFC0F0035
:10439000FDF7F8FDCDE7FDF70BFECAE7DBF80020DF
:1043A000594692060AD50968C1F3C1022AFA02F1F8
:1043B000626A36F81220B1FBF2F20FE0616A36F859
:1043C0001120BAFBF2F209E0616A36F811200949BE
:1043D000F1E7616A36F81110B2FBF1F2616802EBA5
:1043E0005102B2FBF1F189B2C16007B03846BDE8B5
:1043F000F08F000000093D0090F87910212901D0CC
:1044000002207047B0F8621021B18168B1F5805F79
:1044100013D014E001680A68920004D58A6822F477
:1044200000028A6003E00A6822F080020A600068E5
:10443000016841F0400101600CE0016961B1C16DAA
:104440004A1CC265026809781185B0F86210491EDD
:10445000A0F8621000207047C16D02680988C1F39E
:1044600008011185C16D891CC165EEE72DE9F04198
:104470001E46174688460446069D1CE0681C1AD056
:1044800025B1FCF72FFE801BA84214D920680168D3
:1044900021F4D07101602068816821F00101816000
:1044A000202084F8790084F87A00002084F87800CD
:1044B0000320BDE8F0812068C16938EA010004D01A
:1044C0000020B842DAD00020F3E70120F9E700002D
:1044D00070B50D4D00240D48FEF720FB02E0641C72
:1044E000AC4204D80948FEF713FB2028F7D100247A
:1044F00002E0641CAC4206D8054901220348FEF7DD
:1045000043FC0028F5D170BDFFFF0100F800002436
:1045100018000024FEE70907090E002804DB00F15B
:10452000E02080F80014704700F00F0000F1E02058
:1045300080F8141D704702E008C8121F08C1002A45
:10454000FAD170477047002001E001C1121F002A14
:10455000FBD1704710B504460420FEF7B7FA0148B6
:10456000046010BD1400002470B5002405464FF40B
:104570007A7603E0304600F005F8641CAC42F9D3CB
:1045800070BD000070B54FF0E02500216C69094A4C
:10459000AB6912685043AA699A42FCD002D2A3EBDD
:1045A000020302E0A4EB020633441944134681429D
:1045B000F1D370BD1400002408B5FBF7EDFEFCF745
:1045C0009FFD042302220521A020FFF741FB4FF4A9
:1045D000C870FFF7BFFF4FF4E13000F0DFF8FEF7DF
:1045E000ABFFFEF753FCFEF7C9FFFEF7B5FDFCF786
:1045F000A1F94FF6FF752846FEF7BAFC10214FF4DB
:104600007846084631A33246FBF772FF1F2220216D
:10461000102034A3FBF76CFF1F223021102037A39A
:10462000FBF766FF1F22462110203AA3FBF760FF2D
:104630003E4F3F4C0020FEF759FC0128207018D156
:10464000EF2240F23F135A2100950020FEF70EFDA5
:104650001F225A21102037A3FBF74AFF3B490522AE
:104660003846FFF7DBF91F225A21102038A3FBF749
:104670003FFF2078022818D11F225A2110203AA388
:10468000FBF736FF2A4905223846091DFFF7BCF91A
:104690001F225A2110203AA3FBF72AFF244B6E2138
:1046A000102032461B1DFBF723FF6088401C6080F2
:1046B0000A20FFF759FF60881428BBD13648022131
:1046C000FCF707FD00206080B4E7000053544D3331
:1046D00032483720464C4153482D454550524F4DA6
:1046E000200000002020C7B6C8EBCABDBFAAB7A2F1
:1046F000CDF8202020202020200000006D6375646C
:1047000065762E74616F62616F2E636F6D2020205D
:1047100020000000204B313A577269746520204B0D
:10472000323A5265616420202000000000800008B9
:1047300000000024537461727420577269746520FC
:10474000464C4153482E2E2E2E000000D447000820
:10475000464C4153482057726974652046696E691A
:10476000736865642100000053746172742052659F
:10477000616420464C4153482E2E2E2E200000000E
:1047800054686520446174612052656164656420E9
:1047900049733A2020000000000002580B490A4AE1
:1047A00010B5C1E9002000208860C86008618861F8
:1047B0000C2048610846FEF771FABDE81040044934
:1047C00001220248FEF7E0BA00100140F800002480
:1047D0001800002453544D333220464C4153482096
:1047E0005445535400000000000102030401020379
:1047F0000406070809000100020004000600080082
:104800000A000C00100020004000800000010000A1
:1048100000000000000000000000000000003F4019
:1048200000000000000000003000400030004000A8
:10483000000009000BC03D000BC03D00090018C07E
:1048400024407FE0224031800000180024C01B007B
:104850000D803240018003801C4027401C800740AF
:104860000040100060000000000000000000000098
:10487000000000001F802040402000004020204019
:104880001F8000000000090006001F8006000900CC
:104890000000040004003F80040004000000001039
:1048A000006000000000000000000400040004009C
:1048B00004000400000000000040000000000000B0
:1048C0000000002001C006003800400000001F80EA
:1048D0002040204020401F800000000010403FC0CA
:1048E00000400000000018C0214022402440184031
:1048F000000010802040244024401B800000020063
:104900000D0011003FC0014000003C8024402440C5
:104910002440238000001F80244024403440038032
:1049200000003000200027C03800200000001B805D
:104930002440244024401B8000001C0022C0224050
:1049400022401F800000000000000840000000001E
:1049500000000000000004600000000000000000F3
:1049600004000A00110020804040090009000900ED
:1049700009000900000000004040208011000A00EA
:1049800004001800200023402400180000001F80AD
:104990002040274029401F400000004007C0390048
:1049A0000F0001C0004020403FC0244024401B8035
:1049B00000001F8020402040204030800000204028
:1049C0003FC0204020401F80000020403FC02440C6
:1049D0002E4030C0000020403FC024402E00300058
:1049E00000000F0010802040224033800200204051
:1049F0003FC0040004003FC02040204020403FC092
:104A00002040204000000060202020203FC02000E7
:104A1000200020403FC024400B0030C020402040F8
:104A20003FC020400040004000C03FC03C0003C0E9
:104A30003C003FC0000020403FC00C4023003FC06E
:104A400020001F802040204020401F800000204088
:104A50003FC024402400180000001F802140214056
:104A600020E01FA0000020403FC02440260019C0C5
:104A7000004018C024402440224031800000300013
:104A800020403FC020403000000020003F80004018
:104A900000403F80200020003E0001C00700380099
:104AA0002000380007C03C0007C03800000020404C
:104AB00039C0060039C0204000002000384007C03F
:104AC000384020000000304021C02640384020C03F
:104AD0000000000000007FE04020402000000000B7
:104AE00070000C00038000400000000040204020C7
:104AF0007FE00000000000002000400020000000D7
:104B00000000001000100010001000100010000045
:104B1000000040000000000000000000028005408E
:104B2000054003C0004020003FC004400440038013
:104B30000000000003800440044006400000000024
:104B40000380044024403FC0004000000380054033
:104B5000054003400000000004401FC024402440E2
:104B60002000000002E005500550065004202040BF
:104B70003FC00440040003C000400000044027C0C0
:104B800000400000000000100010041027E00000AA
:104B9000000020403FC00140070004C00440204006
:104BA00020403FC000400040000007C0040007C094
:104BB000040003C00000044007C00440040003C018
:104BC0000040000003800440044003800000041003
:104BD00007F00450044003800000000003800440FC
:104BE000045007F00010044007C002400400040015
:104BF0000000000006400540054004C00000000021
:104C000004001F80044000400000040007800040B2
:104C1000044007C000400400070004C001800600F3
:104C20000400060001C0070001C0060000000440A7
:104C300006C0010006C0044000000410071004E094
:104C40000180060004000000044005C00640044046
:104C500000000000000004007BE040200000000095
:104C600000000000FFF000000000000040207BE09A
:104C700004000000000040008000400020002000F0
:104C800040000000000000000000000000000000E4
:104C900000000000000000001FCC000C000000001D
:104CA00000000000080030006000080030006000D4
:104CB0000000022003FC1E20022003FC1E20022014
:104CC000000000000E1811043FFF10840C78000053
:104CD00000000F0010840F3800C007781884007897
:104CE000000000780F8410C411240E9800E40084A2
:104CF00000080800680070000000000000000000CC
:104D0000000000000000000007E018182004400226
:104D10000000000040022004181807E00000000016
:104D200000000240024001800FF00180024002407A
:104D300000000080008000800FF80080008000806C
:104D400000000001000D000E000000000000000047
:104D50000000000000800080008000800080008053
:104D600000800000000C000C0000000000000000AB
:104D70000000000000060018006001800600180016
:104D80002000000007F0080810041004080807F0CD
:104D900000000000080408041FFC000400040000D8
:104DA000000000000E0C10141024104411840E0C8E
:104DB000000000000C1810041104110412880C707B
:104DC0000000000000E00320042408241FFC00244D
:104DD000000000001F981084110411041088107046
:104DE0000000000007F00888110411041888007002
:104DF000000000001C00100010FC13001C0010003C
:104E0000000000000E3811441084108411440E3844
:104E1000000000000700088C10441044088807F0C8
:104E20000000000000000000030C030C0000000064
:104E3000000000000000000101060000000000006A
:104E40000000000000800140022004100808100447
:104E50000000022002200220022002200220022064
:104E60000000000010040808041002200140008027
:104E7000000000000E001200100C106C10800F00DB
:104E8000000003E00C1813E4142417C4082807D00A
:104E900000000004003C03C41C40074000E4001C68
:104EA000000410041FFC1104110411040E8800708A
:104EB000000003E00C1810041004100410081C106B
:104EC000000010041FFC100410041004080807F070
:104ED000000010041FFC1104110417C4100408186A
:104EE000000010041FFC1104110017C0100008007E
:104EF000000003E00C181004100410441C7800405B
:104F0000000010041FFC10840080008010841FFC2F
:104F100010040000100410041FFC10041004000012
:104F2000000000030001100110011FFE100010001E
:104F3000000010041FFC110403801464181C1004EA
:104F4000000010041FFC1004000400040004000C06
:104F5000000010041FFC1F0000FC1F001FFC1004B9
:104F6000000010041FFC0C04030000E010181FFCDC
:104F7000100007F00808100410041004080807F0D7
:104F8000000010041FFC10841080108010800F009F
:104F9000000007F0081810241024101C080A07F25B
:104FA000000010041FFC1104110011C011300E0C80
:104FB000000400000E1C11041084108410441C38DE
:104FC00000001800100010041FFC1004100018004E
:104FD000000010001FF810040004000410041FF863
:104FE000100010001E0011E0001C007013801C0057
:104FF00010001FC0103C00E01F0000E0103C1FC06C
:1050000000001004180C163401C001C01634180C2E
:10501000100410001C00130400FC13041C001000FA
:1050200000000804101C1064108413041C041018E1
:1050300000000000000000007FFE4002400240022D
:105040000000000030000C0003800060001C000322
:10505000000000004002400240027FFE000000000D
:105060000000000000002000400040004000200040
:105070000000000100010001000100010001000129
:10508000000100004000400020000000000000007F
:10509000000000000098012401440144014400FC88
:1050A000000410001FFC0088010401040088007047
:1050B0000000000000700088010401040104008861
:1050C00000000000007000880104010411081FFCAA
:1050D0000004000000F8014401440144014400C8F8
:1050E00000000000010401040FFC11041104110070
:1050F0001800000000D601290129012901C9010673
:10510000000010041FFC008401000100010400FCE9
:10511000000400000104190419FC0004000400004C
:1051200000000000000300010101190119FE000048
:10513000000010041FFC0024004001B4010C010415
:1051400000000000100410041FFC00040004000014
:105150000000010401FC0104010001FC0104010044
:1051600000FC010401FC008401000100010400FCBA
:105170000004000000F8010401040104010400F827
:105180000000010101FF0085010401040088007096
:10519000000000000070008801040104010501FF07
:1051A00000010104010401FC0084010401000180EC
:1051B0000000000000CC01240124012401240198F6
:1051C000000000000100010007F8010401040000D4
:1051D0000000010001F8000400040004010801FCC3
:1051E0000004010001800170000C001001600180CA
:1051F000010001F0010C003001C00030010C01F091
:10520000010000000104018C00740170018C010494
:105210000000010101810171000E00180160018090
:10522000010000000184010C013401440184010CDF
:105230000000000000000000000001003EFC4002F1
:1052400040020000000000000000FFFF000000001E
:1052500000000000400240023EFC0100000000008F
:10526000000000006000800080004000400020003E
:10527000200000000000000000000000000000000E
:10528000000000000000000000000000000000001E
:10529000000000000000000000000000000000000E
:1052A00000000000000F80380FFE380F803800002B
:1052B00000000000000000000000000000000000EE
:1052C0000100000600000C0000380000310000065C
:1052D00000000C000038000030000000000000005A
:1052E000000061800067F807F9800061800061803C
:1052F0000061800061800067F807F980006180002C
:10530000000000000000000001C0E003E0F00630F3
:10531000080418081FFFFE040E080787F00381E049
:1053200000000000000001F000060C000404080664
:105330000C7001F9C0000E00003BE000EC180708FB
:1053400008040C180003E00000000001E00007F072
:1053500003F818041C0804170807E1D003C0E00094
:1053600023B0003C080020080000100000000000EE
:10537000000100003100003200001C0000000000AD
:10538000000000000000000000000000000000001D
:10539000000000000000000000000000000000000D
:1053A00000007F0001FFC00780F00C00181000040F
:1053B0002000020000000000002000021000040C89
:1053C00000180780F001FFC0007F0000000000000F
:1053D000000000000000000000000000000042008B
:1053E000006600006600003C0000180003FFC000DB
:1053F0001800003C0000660000660000420000004B
:105400000000080000080000080000080000080074
:1054100001FFC000080000080000080000080000AC
:105420000800000000000001000031000032000010
:105430001C00000000000000000000000000000050
:10544000000000000000000000000800000800004C
:10545000080000080000080000080000080000081C
:10546000000008000008000000000000000000002C
:105470000000380000380000380000000000000084
:10548000000000000000000000000000000000001C
:105490000000000600001C000070000180000E00EB
:1054A00000380000C0000700001C000030000000B1
:1054B0000000000000007F8001FFE0038070060014
:1054C0001804000804000806001803807001FFE0BB
:1054D000007F8000000000000000000001000801C3
:1054E000000801000803FFF807FFF80000080000AB
:1054F0000800000800000000000000000001C038A3
:1055000002C0580400980401180402180404180684
:105510001C1803F81801E0F800000000000000006B
:105520000001C0E003C0F0040008040808040808F3
:1055300006180803F41801E7F00001E0000000007D
:105540000000000000000300000D000011000061D9
:105550000000810803010807FFF80FFFF8000108A9
:105560000001080000000000000000E007FCD00679
:105570000808061008061008061008061838060F56
:10558000F00607C0000000000000000000003F809F
:1055900001FFE00384300208180410080410080416
:1055A0001008071810030FF00007C00000000000EB
:1055B0000000000003C0000700000600000600F81D
:1055C0000607F806180006E00007000006000000C5
:1055D000000000000001E1E003F7F00634100418B9
:1055E00008041808040C08040C0806161803F3F045
:1055F00001C1E000000000000000F80003FC3003DF
:10560000063804020804020804020804041003080F
:10561000F001FFC0007F000000000000000000005B
:10562000000000000000000000007038007038002A
:1056300070380000000000000000000000000000C2
:105640000000000000000000000000000000301A10
:1056500000301C00000000000000000000000000FE
:1056600000000000000000000008000014000022FC
:105670000000410000808001004002002004001072
:1056800008000800000000000000210000210000C8
:105690002100002100002100002100002100002144
:1056A00000002100002100000000000000000000B8
:1056B0000800080400100200200100400080800063
:1056C000410000220000140000080000000000005B
:1056D0000003C00004C000040000080038080F38B0
:1056E0000808380810000C300007E00003C0000074
:1056F0000000000000003F8000FFE0038070020F08
:105700001006708804C088048308047F8802C09053
:1057100003012000FE400000080000180001F8000E
:105720003E0801C20007020007E20000FE00001F61
:10573000C80001F800003800000804000807FFF85E
:1057400007FFF80408080408080408080408080605
:10575000180803F41801E7F00001E0000000000061
:1057600000003F8001FFE003807002001804000881
:105770000400080400080400100600200780C00090
:10578000000004000807FFF807FFF8040008040001
:105790000804000804001802001003807001FFE0F4
:1057A000007F8000000004000807FFF807FFF804EE
:1057B0000808040808040808040808043E0804004F
:1057C0000806001801006000000004000807FFF848
:1057D00007FFF8040808040800040800040800048F
:1057E0003E000600000600000180000000000000EE
:1057F00000003F8001FFE0038070060018040008ED
:105800000402080402080203F00783F0000200000B
:10581000020004000807FFF807FFF8040808000862
:105820000000080000080000080004080807FFF84E
:1058300007FFF8040008000000000000040008044E
:10584000000804000807FFF807FFF8040008040038
:10585000080400080000000000000000000000062E
:105860000000070000010400010400010400030718
:10587000FFFE07FFFC040000040000040000040019
:105880000807FFF807FFF8040C08001800003E00A6
:1058900004C7800503C80600F80400380400180097
:1058A000000804000807FFF807FFF80400080000DC
:1058B00008000008000008000008000008000018A8
:1058C00000006000000004000807FFF807800807D8
:1058D000FC00007FC00003F80007C00078000780CC
:1058E0000807FFF807FFF804000804000807FFF89E
:1058F00007000803C00000E000003800001E0000A0
:1059000007000001C00400F007FFF80400000000D9
:1059100000007F8001FFE00380700600180400088B
:1059200004000806001803003001FFE0007F80003B
:10593000000004000807FFF807FFF8040408040447
:1059400000040400040400040400060C0003F80032
:1059500001F000000000000000007F8001FFE00374
:1059600080700600880400880400C806003C03001C
:105970003E01FFE6007F8400000004000807FFF8F6
:1059800007FFF8040808040800040C00040F0004D2
:105990000BC00610F003F03801E00800000800001A
:1059A0000001E0F803F0300630100418080418086D
:1059B000040C08040C080206180207F00781E00036
:1059C0000000018000060000040000040000040044
:1059D0000807FFF807FFF8040008040000040000AF
:1059E00006000001800004000007FFE007FFF0044C
:1059F000001800000800000800000800000800006F
:105A00000804001007FFE004000004000006000086
:105A100007E00007FE00041FE00001F80000380066
:105A200001E0043E0007C00006000004000004007E
:105A30000007E00007FFC0041FF80007C007F800D8
:105A400007FF80043FF80007C004F80007000004C7
:105A5000000000000004000806001807C07805F1E7
:105A6000C8003E00001F800463E80780F8060018A5
:105A70000400080000000400000600000780000782
:105A8000E008047C08001FF80007F800180804E08C
:105A900008070000060000040000000000010008E4
:105AA0000600380400F80403E8040F08047C080525
:105AB000F00807C00807001804006000000000009C
:105AC000000000000000000000000000003FFFFE9A
:105AD000200002200002200002200002200002001C
:105AE000000000000000000008000007000000C0E7
:105AF000000038000006000001C000003000000E69
:105B00000000010000000000000000002000022052
:105B100000022000022000022000023FFFFE0000E1
:105B20000000000000000000000000000000000075
:105B300000000008000010000030000020000030CD
:105B4000000010000008000000000000000000003D
:105B5000010000010000010000010000010000013F
:105B60000000010000010000010000010000010030
:105B700000010000000000000000002000002000E4
:105B800000100000100000000000000000000000F5
:105B90000000000000000000000000F00019F80004
:105BA0001B18002208002608002408002410003FCB
:105BB000F8001FF8000008000018000000040000B2
:105BC00007FFF80FFFF00018180010080020080069
:105BD0002008003018001FF0000FC0000000000077
:105BE000000007C0001FF000183000200800200847
:105BF000002008003C08001C1000006000000000AD
:105C000000000000000007C0001FF000381800204E
:105C10000800200800200804101007FFF80FFFF00C
:105C20000000100000000000000000000007C0009D
:105C30001FF0001230002218002208002208003253
:105C400008001E10000E20000000000000002000D0
:105C500000200800200801FFF803FFF806200804D0
:105C600020080420080720000300000000000000B6
:105C70000000000E000E6E001FF30031B10020B1D5
:105C80000020B1003191001F13002E1E00200E00D5
:105C9000300000000004000807FFF80FFFF80010B4
:105CA00008002000002000002008003FF8001FF836
:105CB00000000800000000000000000000200800B4
:105CC0002008002008063FF8063FF8000008000002
:105CD00008000008000000000000000000000000B4
:105CE0000000030000030020010020010020030643
:105CF0003FFE063FFC000000000000000000000026
:105D00000004000807FFF80FFFF8000188000300F7
:105D1000002FC00038F800203800200800000800DC
:105D20000000000000000000040008040008040057
:105D30000807FFF80FFFF80000080000080000083F
:105D4000000000000000002008003FF8003FF800BD
:105D50001008002000003FF8003FF8001008002065
:105D600000003FF8003FF800000800000000200895
:105D7000003FF8003FF8001008001000002000006D
:105D80002008003FF8001FF8000008000000000095
:105D9000000007C0000FF000183000300800200895
:105DA000002008003008001830000FF00007C00085
:105DB0000000000000002001003FFF003FFF001036
:105DC00011002009002008002008003038001FF0D2
:105DD000000FC00000000000000007C0001FF0001E
:105DE0003818002008002008002009001011001FAA
:105DF000FF003FFF00000100000000200800200815
:105E0000002008003FF8003FF800080800100800D4
:105E100020080020000030000030000000000000DA
:105E200000000000000C78001E1800330800230852
:105E30000021080021880021980030F0003860001F
:105E4000000000000000200000200000200000FFF3
:105E5000F003FFF8002008002008002008000030B0
:105E6000000000000000000000002000003FF000E3
:105E70007FF8000018000008000008002010003F14
:105E8000F8007FF00000100000000000000020007B
:105E9000003000003C00003F800023F0000078004C
:105EA0000070002380003C00003000002000002033
:105EB00000003C00003FE00023F80000E000270065
:105EC000003E00003FE00021F80001E0003E00003D
:105ED0002000000000002008002008003838003EA4
:105EE000680027800003C8002CF80038380020180C
:105EF0000020080000000000000020000030030027
:105F00003C01003F830023EC000070002380003C34
:105F10000000200000200000000000000000000041
:105F20000038080020380020F80023E8002F8800FF
:105F30003E08003808002018000070000000000033
:105F40000000000000000000000000000000080049
:105F50000014001FF7FC30000620000200000000C3
:105F60000000000000000000000000000000000031
:105F700000000000FFFFFF00000000000000000024
:105F800000000000000000000000000020000230BF
:105F900000061FF7FC0014000008000000000000CD
:105FA00000000000000000000000000000180000D9
:105FB00060000040000040000020000010000008C9
:105FC00000000400000400000C0000100000B5E711
:105FD0000200020002007FF0421042107FF04210E7
:105FE00042107FF042000208020801F800000000A1
:105FF000D7D37FF000200040008001000200FFF8AE
:106000000200020002000200020002000E00000076
:106010000000BCBC10201020102013FEFC2010201B
:10602000102015FC18843088D048105010201050D3
:1060300051882606CAF501000120011001107FFCDD
:106040000380054005400920111021084104010288
:10605000010001000100D2BA0080404027F8114041
:1060600001408278424816A81AD0235022204220AC
:106070004250028800000000BEA73FE020203FE021
:1060800020203FE00000FDF885088508FDF8850820
:106090008508FDF8850800000000B2E200084F887E
:1060A00028880AA88AA84AA80AA82AA82AA84228AA
:1060B000450884888888103800000000CAD4405001
:1060C000204820400FF80040E04027402240224076
:1060D00022202A2833A82E18000800000000B3CC84
:1060E00000001BF0E210221023F0F800200033F033
:1060F00068806080A3F02080208027F800000000E6
:10610000D0F2020001003FF820002FF020202240B2
:1061100021803FF8208820904080408083800000CC
:106120000000D1D5200010F87E20444028F87E8859
:1061300048A850A864A848A872A884501888610884
:1061400000000000C9AB100010003FE0404080801C
:106150007FF04210421042107FF04000400840089B
:106160003FF800000000CCEE20802FF8208027F0C0
:10617000F41027F0241027F0241027F03410CFF863
:106180000220041000000000B3E404000200FFF845
:106190000800104020207FF00890088008800880C8
:1061A00010882088C07800000000CEC404000200DF
:1061B0000200FFF81040104008800880050002002F
:1061C000050008803060C01800000000D7D6040029
:1061D0000200FFF8800880083FC000800100020034
:1061E000FFF80200020002000E0000000000CFD401
:1061F0003FE0202020203FE0202020203FE00880BA
:106200004890289028A008800880FFF8000000002F
:10621000CABE00003FE0000000000000FFF80200DE
:106220001240122022104208820802000E000000D4
:106230000000CDBC7FF84008440847C8484854884F
:1062400043084CC8733840884C08430840887FF89E
:1062500000000000C6AC00802080208020803FF03D
:106260002000200020003FC020402040204040402F
:10627000804000000000B4A520403840484091F024
:106280007D50555055507D5055F054407C405450F1
:1062900057F88C0800000000C3FE2220222027F8B7
:1062A000FA2027F0241027F03410E7F020802FF890
:1062B00021402220EC1800000000CAE44080414048
:1062C000F22044108BE8A000F78824A827A834A85F
:1062D000E7A824A8248825B800000000C8EB08001F
:1062E0000400040002000200050005000880088088
:1062F0001040104020204010800800000000C8AB73
:10630000020002000500088010402020DFD80200B3
:1063100002001FC0020002000200FFF8000000009F
:10632000B3CC00001BF0E210221023F0F800200094
:1063300033F068806080A3F02080208027F8000080
:106340000000BCBC208020802080F7F020802080CE
:1063500027E03220E2202140208021402220EC183A
:1063600000000000CAF50200024002200200FFF80F
:1063700007000A800A801240222042108208020090
:10638000020000000000D6A702000200FFF8020091
:1063900002007FE010201040088005000200050088
:1063A00018C0E03800000000B3D62080208023F021
:1063B000F880208027F828203020E7F820202220AD
:1063C00021202020E0E000000000D7A80200020009
:1063D0007FF004000400FFF8080010003FE00020F8
:1063E00000401C800300008000000000D7A20100D4
:1063F0004080200017F0008080804080008017F0EF
:1064000010802080208040804FF800000000C5FAF6
:10641000204024402440F448245027602440344045
:10642000E4402440244025482648E4380000000089
:10643000B7A202002220221044007FF804000800C6
:106440000FE0142024404280810006C0383800004C
:106450000000B3C900A0009000807FF84080409009
:106460007C90449044A044A0444858A84118820815
:1064700000000000B9A601000100F90023F021107E
:1064800021102110211021103910C2100210041007
:10649000086000000000D2C60000002000780CE474
:1064A0007904516810307E6019981A3C2FE448E452
:1064B0000838003000600000D1A100000120012058
:1064C00003FC62203420042003FC240021B021209E
:1064D0002220323E18000FE00000D4F1000000003E
:1064E00010FC1304110C3DF8703E10D015907CF098
:1064F000503E18101BFE023000200000CFEE0000BE
:10650000000003FE00607C4012FC110411061136ED
:1065100011241F44794400C0009C01860000C4BFC0
:10652000000000000FE03C18200820043E04600436
:1065300060047E046004200C20081FF0018000002D
:10654000B6CC0000080011FC103E3EF82D8C29044A
:10655000490409043E8C50FC10881EC811FC100E22
:106560000000B0B400000040006012FE13023A4286
:106570007F4410C41BFE3C987190113011A000782C
:10658000004C0000C8B70000004000F878C41F8C21
:10659000313821EC2126413A7DE2272225FA3D2699
:1065A000012401040000B6A80000010001705FFC96
:1065B000700420042FF801001100113821C43100AB
:1065C0003F0063E040380000B3A40000000008185A
:1065D000086008C00B001E00181C7FF0100011801E
:1065E00010E01838098E0F000000B0B40000004021
:1065F000006012FE13023A427F4410C41BFE3C9816
:106600007190113011A00078004C0000B7B5000067
:10661000000007F80600240014F8078C040424087E
:10662000261825F0647C64C220801FC00000BBD8FF
:10663000000000001FF030182008278C2C4428444C
:1066400028442CC427842004300C1FF80380000049
:10665000C7B60100210821083FF800202220223E71
:10666000FF42229422103E10221022283E2822446B
:106670000082CABD0048004400440040FFFE0040C4
:1066800000403E4008400840082008220F12780AC7
:1066900020060002BFAA00007FFC08200820082076
:1066A00008200820FFFE08200820082008201020CD
:1066B000102020204020B7A2010011101108220054
:1066C0003FFC0200040007F80A080908111010A096
:1066D000204040A003181C06CDF800007FFC4004B9
:1066E0004004421452944A54442444244A544A5480
:1066F00052946104400440144008D6D001000100C7
:10670000010001003FF82108210821082108210883
:106710003FF821080100010001000100CEC4020081
:1067200001000100FFFE1010101008200820044096
:10673000028001000280044008203018C006B2E246
:10674000000427C414441454855445544554155426
:1067500015542554E55421042284224424140808A5
:10676000CAD4002820241024102007FE0020F02086
:1067700017E0112011101110151019CA170A02067E
:106780000002000000000000000000000000000007
:1067900000000000000000000000000000000000F9
:1067A00000000000B4F3000000000000001800002A
:1067B000100000100000100000100000100C3FFF3F
:1067C000FE00100000180000180000340000340023
:1067D00000220000620000410000C1800080C00172
:1067E000006006003808001C300000000000D4BD26
:1067F0000000000000000300C00200B00200980288
:1068000060881F888C020FF0020C80022C887FDCCD
:1068100088030C901B0CD01B0C6013EE60131E64DD
:10682000130CF413019C1B020C27040421D8004014
:106830007FFC4007F8000000B4B400000000000036
:1068400003800803000C02E00C06300C04198C08CD
:10685000088C08008C18208C2FF08C48208C082085
:106860008C08208C08208C08608C09C10C08080C4E
:1068700008080C08080C0C0C0C07FC780000100031
:106880000000D0C200000000000002000801003C2F
:106890000133C03EC20008620004420004820004CA
:1068A0009A0C3FFFFE0102300102300112301FE25C
:1068B000300102300D4230193630111430211430BD
:1068C000210830471030022030000000D2BA00000A
:1068D000000000000006001803000C020C04FDF08C
:1068E0000119800111004233083222F812421812B5
:1068F000651004E490056AB0056A200A71200861F9
:10690000403860C01860C018616018623018641E9A
:10691000087800000000BEA7000000000000010091
:106920004001FFC001004001004001FFC0010040E4
:1069300001004001FFC00100400000001064081F7A
:10694000E7F81046081046081046081FC7F810461A
:10695000081046081046081FC7F810460800000037
:10696000C6C10000000000000800000FFFF80C0086
:10697000180C00180FFFF80C40900C30C00C108061
:106980000C11100DFFF8083080083080083088089E
:10699000309C1FFFE010208010208020608020406D
:1069A00080408080030080000000B2E20000000010
:1069B000000011000C09FE080D860805864801A696
:1069C0004841B64833B64813B64815B64805B648E8
:1069D00005B64805B64809A64809A64839A4481886
:1069E0002048185808184408188608190238060064
:1069F00018000000CAD40000000000000001A01030
:106A000001D80800880C008804008400FFFE000004
:106A1000800000800400803C0280047DC00408C027
:106A2000040840040840044860048822050F340725
:106A3000381406E01C04000E0000060000000000F0
:106A40000000000000000000000000000000000046
:106A50000000000000000000000000000000000036
:106A60000000000000000000000000000000000026
:106A70000000000000000000000000000000000016
:106A80000000000000000000A86A000800000024C8
:106A90003000000036450008D86A000830000024A5
:106AA000000C000046450008000000000000000047
:106AB000000000000090D0030090D0030000000010
:106AC00000000000010000001000000000000000B5
:086AD00001000000FFFF0000BF
:040000050800029954
:00000001FF
